:020000040000FA
:100000002E288207003400340034003400341B34BE
:1000100077344034003435346734E03400346A34A3
:10002000CF34C03400349A341D3420340034D534F5
:100030009F34803401341334B234203401344034DA
:100040006F34403401347B34CA3490340134AB34DF
:100050003F3400340134C934C33480348B01073059
:100060009F00A62383168113FB308500860183122F
:100070000511C820E820D110051A4128D114062204
:10008000D11083169B018E231A088312BB0083169E
:100090008E231A088312BC0083168E231A0883123B
:1000A000BD0083168E231A088312BE0083168E238A
:1000B0001A088312A00083168E231A088312A10047
:1000C00083168E231A088312A20083168E231A0821
:1000D0008312A300E42212239322CA22CA22050813
:1000E000CB0003304B05CA00C8014030C700CC012B
:1000F000CF01A321CB197E289E207928B501B40118
:10010000B3010130B2004B1A8F28E830B20003303F
:10011000B3008F280310B20DB30DB40DB50DC70D8C
:10012000C80D031C8A28CC189728902199285321A0
:100130006B21E42212239322CA227928CC18AA2800
:100140000430CF02D7304F07031CA8282830CF0037
:10015000B620B1280430CF07D7304F070318CF019E
:10016000B620E42212239322CA2208004F0801205D
:10017000A300CF0A4F080120A200CF0A4F08012098
:10018000A100CF0A4F080120A0000330CF020800D1
:100190009D230330860006169D2306120330860039
:1001A0000616A0230612033086000616A0230612A8
:1001B000023086000616A323061228305F2308307B
:1001C0005F2301305F2306305F230C305F2308007C
:1001D00080305F23503063234930632343306323EF
:1001E000453063234C3063236730632365306323DA
:1001F0006E3063238830C3005F23363063232E3094
:100200006323303063232D30632336306323303053
:1002100063232030632320306323C0305F234130C9
:10022000632341306323303063235A3063235A30D1
:100230006323203063232F306323203063234B302C
:100240006323613063236E3063236730632361303F
:100250006323203063235530632353306323922379
:10026000C0305F232030632320306323203063239A
:100270002030632320306323203063232030632326
:100280002030632320306323203063232030632316
:100290002030632320306323203063232030632306
:1002A0002030632308003208A007031C5C29A10F3B
:1002B0005C29A20F5C29A30A3308A107031C632948
:1002C000A20F6329A30A3408A207031C6829A30A02
:1002D0003508A3070800FC302307031887290330DB
:1002E0002302031C8F296C302207031887299330BF
:1002F0002202031C8F2978302107031887298730B1
:100300002102031C8F2900302002031C8F2900309A
:10031000A0008730A1009330A2000330A3000800A2
:10032000B209B309B409B509B20F9B29B30F9B29D0
:10033000B40F9B29B50A5321A31FA229A001A10133
:10034000A201A3010800C8014030C700D11CCD2183
:10035000C81BAE290830C7070318C80A0508CB0018
:1003600003304B05C9004A060319A6290310CA0D1C
:100370004908CA064A080239CD004C060319C529A6
:100380004D08CC004908CA00A629CC01CA1CCA29BC
:100390000230CC004908CA000800051ED229851980
:1003A000DB29D7298519D9295118DD29F0295114BC
:1003B000052A5110052AD101052A1030D200051A4C
:1003C000E6299A23D20BDF297A22052AB5010F30BC
:1003D000B4004230B3004030B20053216B21012AF7
:1003E0001030D2008519F9299A23D20BF2297A22EA
:1003F000052AB5010F30B4004230B3004030B200DE
:100400009021E42212239322CA2208008030A00007
:100410009630A1009830A2000030A30083169B0103
:100420008E231A088312BB0083168E231A088312A8
:10043000BC0083168E231A088312BD0083168E23F8
:100440001A088312BE00E4221223C430C3005F23C3
:100450004330C30063234130C30063234C30C300E7
:1004600063239322CA22A321B501B401B301103042
:10047000B2004B193D2A8030B2000000CC184B2A44
:10048000B209B309B409B509B20F4B2AB30F4B2A0D
:10049000B40F4B2AB50A3208BB07031C542ABC0F01
:1004A000542ABD0F542ABE0A3308BC07031C5B2A1A
:1004B000BD0F5B2ABE0A3408BD07031C602ABE0AB2
:1004C0003508BE07051E312A3B0883169B019A009A
:1004D000812383123C0883169A00812383123D08EE
:1004E00083169A00812383123E0883169A00812383
:1004F00083120800831604309B00831220088316A1
:100500009A0081238312210883169A008123831283
:10051000220883169A0081238312230883169A00E7
:10052000812383120800AD01AE01AF01B001B1011A
:100530002030B8003B08BF003C08C0003D08C100A7
:100540003E08C20003103F1CBC2A2008AE07031C53
:10055000AE2AAF0FAE2AB00FAE2AB10A2108AF07FC
:10056000031CB52AB00FB52AB10A2208B007031C34
:10057000BA2AB10A2308B107B10CB00CAF0CAE0C0B
:10058000AD0CC20CC10CC00CBF0CB80BA22A0130C0
:10059000B10008002D3084000008BA000830B9000E
:1005A000BA0C031CD72A861506150611DA2A8611FD
:1005B00006150611B90BD02A840A32300402031C36
:1005C000CC2A8617861308002030B600A801A9019E
:1005D000AA01AB01AC010310A00DA10DA20DA30D4A
:1005E00003182014A80DA90DAA0DAB0DAC0DB60370
:1005F000031DFB2A0800283084000723840A0723F0
:10060000840A0723840A0723840A0723EB2A03307A
:100610000007B700B719800030300007B700B71BDC
:100620008000080080305F23203063232B0E0F39B9
:10063000303E63232B080F39303E63232C30632375
:100640002A0E0F39303E63232A080F39303E6323C8
:10065000290E0F39303E63232E30632388305F2309
:1006600029080F39303E6323280E0F39303E6323AB
:1006700028080F39303E6323203063236B30632317
:10068000483063237A3063232030632308008601D7
:10069000831608308600831206138616FF30C500C5
:1006A00006160608C4000612000000000616000028
:1006B0000612C50303195E2BC419502B0800C30092
:1006C000D0010613662BC30050140617472386017A
:1006D0008316003086008312861206135018061700
:1006E000F0308605430E0F39860406160000061208
:1006F000F030860543080F398604061600000612FE
:1007000008001C158B1355309D00AA309D009C14C9
:100710009C18882B9C171C119B0A08001C141A0893
:100720009B0A0800972397239723972308009A236F
:100730009A230800FF30C500A82B8030C500A82BE5
:100740004030C500A82B2030C500A82B1030C500B4
:0E075000FF30C600C60BAA2BC50BA82B080055
:084000007F007F007F007F00BC
:02400E00213F50
:10420000DE006500DC00170028000100D600000079
:10421000000000000000000000000000000000009E
:10422000000000000000000000000000000000008E
:10423000000000000000000000000000000000007E
:10424000000000000000000000000000000000006E
:10425000000000000000000000000000000000005E
:10426000000000000000000000000000000000004E
:10427000000000000000000000000000000000003E
:10428000000000000000000000000000000000002E
:10429000000000000000000000000000000000001E
:1042A000000000000000000000000000000000000E
:1042B00000000000000000000000000000000000FE
:1042C00000000000000000000000000000000000EE
:1042D00000000000000000000000000000000000DE
:1042E00000000000000000000000000000000000CE
:00000001FF
